:100000000C942A000C943F000C943F000C943F0089
:100010000C943F000C943F000C943F000C943F0064
:100020000C943F000C943F000C943F000C943F0054
:100030000C943F000C943F000C943F000C943F0044
:100040000C943F000C943F000C943F000C943F0034
:100050000C943F0011241FBECFE5D8E0DEBFCDBF1A
:1000600011E0A0E6B0E0E4ECFBE002C005900D92E8
:10007000A439B107D9F70E9496000C94E0050C94BE
:10008000000080E090E0A0E0B0E00BC00196A11D70
:10009000B11D803C27E2920729E0A20720E0B207C9
:1000A000B9F1C89BF3CF1FBC82E08EBD1DBC1CBC48
:1000B00020E030E040E050E011C08CB59DB58156A5
:1000C0009A4E70F42F5F3F4F4F4F5F4F203C87E2B7
:1000D000380789E0480780E05807D1F0C899EDCF8C
:1000E0008CB59DB5A0E0B0E01EBC81362AEE92072B
:1000F00020E0A20720E0B20738F4B695A7959795BF
:1001000087959C01C90108952EEF3FEFC90108951D
:100110002FEF3FEFC901089520E040E050E0CA0111
:100120000197F1F72F5F2A30D1F70895DF92EF9210
:10013000FF920F931F93CF93DF9320E040E050E0B6
:10014000CA010197F1F72F5F2A30D1F780E00E94B2
:10015000A40120E040E050E0CA010197F1F72F5FD1
:100160002A30D1F781E060E00E947C0180E690E0D7
:100170000E94D50180E061E00E944E028CE690E092
:100180000E94D50120E040E050E0CA010197F1F75C
:100190002F5F2A30D1F720E040E050E0CA010197FC
:1001A000F1F72F5F2A30D1F720E040E050E0CA019C
:1001B0000197F1F72F5F2A30D1F720E040E050E0BF
:1001C000CA010197F1F72F5F2A30D1F720E040E014
:1001D00050E0CA010197F1F72F5F2A30D1F720E0F4
:1001E00040E050E0CA010197F1F72F5F2A30D1F7C4
:1001F00081E060E00E947C0155E3F52E40E5E42EAD
:100200003AE6D32E00E010E0D09A8F2D8A95F1F7D0
:10021000D89A8E2D8A95F1F7D8988D2D8A95F1F779
:10022000D0980E944100EC018FEFCF3FD80739F101
:100230008FEFCE3FD80761F180E060E00E944E0270
:10024000BE0180E090E00E946D0320E030E048E6CF
:1002500052E40E946D020E941903DC01CB0164E0AC
:1002600070E00E94E50188E890E00E94D50120E05E
:10027000C8010197F1F72F5F2A30D1F7C5CF80E091
:1002800060E00E944E0288E790E00E94D501BCCF5A
:1002900080E060E00E944E0280E890E00E94D5017C
:1002A000B3CF87B3807F87BB969A939882E08A9575
:1002B000F1F722E035E0C49A822F8A95F1F786B3F0
:1002C0008295807F922F9A95F1F7C498932F9A95F3
:1002D000F1F7C49A922F9A95F1F796B3922F9A95C7
:1002E000F1F7C498932F9A95F1F787FDE4CF96988C
:1002F00087B38F6087BB0895282F662319F1939ADF
:1003000082E08A95F1F7C49A88B3922F92959F70F4
:10031000807F982B98BB95E0892F8A95F1F7C49838
:10032000892F8A95F1F7C49A88B32F70807F822B2A
:1003300088BB892F8A95F1F7C4989A95F1F70E94A6
:10034000510108959398DCCF1F93182F2CE231E0D0
:1003500040E951E0CA010197F1F721503040D1F74F
:1003600087B38F6087BBBC9A8B9A8E9A88B3807F45
:1003700088BBC4989698939881E08A95F1F7C49ABF
:10038000C19A85E0982F9A95F1F7C4988A95F1F76C
:100390000E94510188E260E00E947C01812F8C6004
:1003A00060E00E947C011F910895CF93DF93EC01E0
:1003B0008881882339F061E00E947C012196888140
:1003C0008823C9F7DF91CF910895EF92FF920F93A1
:1003D0001F93DF93CF9300D000D00F92CDB7DEB73D
:1003E0009C018B017E010894E11CF11C85E0F70162
:1003F00011928A95E9F72115310591F0FE013596A4
:10040000C9016AE070E00E9482058083C9016AE048
:1004100070E00E9482059B0131976115710581F79B
:10042000FFEF0F3F1F0749F125E030E0201B310BA4
:1004300025303105B4F4F701E20FF31F8081890103
:100440000F5F1F4FE00EF11E05C0F70181917F0184
:100450000F5F1F4F805D61E00E947C010530110538
:10046000A4F30F900F900F900F900F90CF91DF910A
:100470001F910F91FF90EF9008958981882359F47F
:1004800020E030E02F5F3F4FF701E20FF31F808144
:100490008823C1F3CDCF20E030E0D1CF843150F4B8
:1004A000623049F0633099F0613059F0806860E063
:1004B0000E947C0108958C5E806860E00E947C014F
:1004C000F9CF8064806860E00E947C01F3CF8C5A91
:1004D000806860E00E947C01EDCFA8E1B0E0E3E736
:1004E000F2E00C94B10569837A838B839C832D831E
:1004F0003E834F835887B9E0EB2EF12CEC0EFD1EA6
:10050000CE010196B7010E940A058E010F5E1F4FB2
:10051000CE010596B8010E940A052985223008F40B
:100520007EC03989323010F4B8017CC08A859A893E
:1005300089278A87243011F0223031F4231709F0FB
:100540006EC06CE870E06EC0343039F41D861E86D3
:100550001F86188A1C861B8604C0323021F484E072
:100560008987B7015FC02B853C858B899C89281BB7
:10057000390B3C872B87ED84FE840F851889AD8865
:10058000BE88CF88D88CEA14FB040C051D0540F406
:10059000EE0CFF1C001F111F215030403C872B87A1
:1005A00020E030E040E050E080E090E0A0E0B0E407
:1005B00060E070E0EA14FB040C051D0540F0282BF8
:1005C000392B4A2B5B2BEA18FB080C091D09B69541
:1005D000A79597958795EE0CFF1C001F111F6F5F65
:1005E0007F4F6F31710531F7DA01C9018F77907054
:1005F000A070B07080349105A105B10561F427FDAC
:100600000AC0E114F1040105110529F0205C3F4FF7
:100610004F4F5F4F20782D873E874F87588BBE0105
:10062000675F7F4FCB010E9435046896EAE00C9427
:10063000CD05ACE0B0E0EFE1F3E00C94B9056983DF
:100640007A838B839C83CE010196BE016B5F7F4FC3
:100650000E940A058D81823061F1823050F1843030
:1006600021F48E81882351F12EC02F81388537FDEA
:1006700020C06E812F3131051CF06623F9F023C0B4
:100680008EE190E0821B930B29853A854B855C8532
:1006900004C056954795379527958A95D2F76623D6
:1006A000B1F050954095309521953F4F4F4F5F4F9A
:1006B0000EC020E030E040E050E009C02FEF3FEFF7
:1006C0004FEF5FE704C020E030E040E050E8B901C0
:1006D000CA012C96E2E00C94D505A8E0B0E0E3E76F
:1006E000F3E00C94B1057B018C0161157105810566
:1006F000910519F482E0898360C083E089838EE1EB
:10070000C82ED12CDC82CB82ED82FE820F8318872B
:10071000C801B7010E94E603FC013197F7FF3BC017
:10072000222733272E1B3F0B57016801022E04C0DE
:10073000D694C794B794A7940A94D2F740E050E0B7
:1007400060E070E081E090E0A0E0B0E004C0880FDD
:10075000991FAA1FBB1F2A95D2F70197A109B109BA
:100760008E219F21A023B1230097A105B10521F07F
:1007700041E050E060E070E04A295B296C297D2966
:100780004D835E836F8378878EE190E08E1B9F0B95
:100790009C838B8312C0309781F00E2E04C0EE0C28
:1007A000FF1C001F111F0A94D2F7ED82FE820F83F7
:1007B0001887CE1ADF0ADC82CB821A82CE0101961C
:1007C0000E9435042896EAE00C94CD05EF92FF9242
:1007D0000F931F937B018C0180E0E81680E0F80600
:1007E00081E0080780E0180788F48FEFE816F1042D
:1007F0000105110531F028F088E090E0A0E0B0E0BC
:1008000017C080E090E0A0E0B0E012C080E0E81601
:1008100080E0F80680E0080781E0180728F088E10A
:1008200090E0A0E0B0E004C080E190E0A0E0B0E0A3
:1008300020E230E040E050E0281B390B4A0B5B0B14
:1008400004C016950795F794E7948A95D2F7F701B7
:10085000EC56FF4F8081281B310941095109C9011C
:100860001F910F91FF90EF900895DF92EF92FF920A
:100870000F931F93FC01E480F58006811781D180DE
:100880008081823048F480E090E0A0E1B0E0E82A86
:10089000F92A0A2B1B2BA5C0843009F49FC0823093
:1008A00021F4EE24FF24870105C0E114F1040105C1
:1008B000110519F4E0E0F0E096C0628173819FEFCA
:1008C000623879070CF05BC022E83FEF261B370B3C
:1008D0002A3131052CF020E030E040E050E02AC021
:1008E000B801A701022E04C07695679557954795E4
:1008F0000A94D2F781E090E0A0E0B0E004C0880F55
:10090000991FAA1FBB1F2A95D2F70197A109B10908
:100910008E219F21A023B1230097A105B10521F0CD
:1009200081E090E0A0E0B0E09A01AB01282B392BE8
:100930004A2B5B2BDA01C9018F779070A070B070E1
:1009400080349105A105B10539F427FF09C0205C69
:100950003F4F4F4F5F4F04C0215C3F4F4F4F5F4FA2
:10096000E0E0F0E02030A0E03A07A0E04A07A0E491
:100970005A0710F0E1E0F0E079018A0127C0603801
:10098000710564F5FB01E158FF4FD801C7018F776E
:100990009070A070B07080349105A105B10539F454
:1009A000E7FE0DC080E490E0A0E0B0E004C08FE37B
:1009B00090E0A0E0B0E0E80EF91E0A1F1B1F17FF31
:1009C00005C016950795F794E794319687E016953C
:1009D0000795F794E7948A95D1F705C0EE24FF2494
:1009E0008701EFEFF0E06E2F679566276795902FF0
:1009F0009F77D794DD24D7948E2F8695492F462B49
:100A0000582F5D29B701CA011F910F91FF90EF90F8
:100A1000DF900895FC01DB01408151812281622F2A
:100A20006F7770E0221F2227221F9381892F880F62
:100A3000822B282F30E0991F9927991F11969C939C
:100A4000119721153105A9F541155105610571056C
:100A500011F482E037C082E89FEF13969C938E9347
:100A600012979A01AB0167E0220F331F441F551FF5
:100A70006A95D1F783E08C930DC0220F331F441F7A
:100A8000551F12968D919C911397019713969C93E5
:100A90008E931297203080E0380780E0480780E48A
:100AA000580758F314962D933D934D935C931797E5
:100AB00008952F3F310579F4411551056105710500
:100AC00019F484E08C93089564FF03C081E08C9353
:100AD00012C01C9210C02F57304013963C932E9397
:100AE000129783E08C9387E0440F551F661F771F92
:100AF0008A95D1F7706414964D935D936D937C93B2
:100B00001797089597FB092E07260AD077FD04D082
:100B10000CD006D000201AF4709561957F4F08958F
:100B2000F6F7909581959F4F0895AA1BBB1B51E145
:100B300007C0AA1FBB1FA617B70710F0A61BB70B4D
:100B4000881F991F5A95A9F780959095BC01CD01F2
:100B500008952F923F924F925F926F927F928F9261
:100B60009F92AF92BF92CF92DF92EF92FF920F933C
:100B70001F93CF93DF93CDB7DEB7CA1BDB0B0FB646
:100B8000F894DEBF0FBECDBF09942A883988488803
:100B90005F846E847D848C849B84AA84B984C88499
:100BA000DF80EE80FD800C811B81AA81B981CE0F90
:100BB000D11D0FB6F894DEBF0FBECDBFED01089575
:040BC000F894FFCFD7
:100BC400556C74726120536F6E69630053656E7364
:100BD4006F722054657374004572726F7220210025
:100BE400436C65617220210020636D0000000000E9
:100BF40000000000000102020303030304040404D0
:100C04000404040405050505050505050505050594
:100C14000505050506060606060606060606060674
:100C24000606060606060606060606060606060660
:100C34000606060607070707070707070707070744
:100C44000707070707070707070707070707070730
:100C54000707070707070707070707070707070720
:100C64000707070707070707070707070707070710
:100C740007070707080808080808080808080808F4
:100C840008080808080808080808080808080808E0
:100C940008080808080808080808080808080808D0
:100CA40008080808080808080808080808080808C0
:100CB40008080808080808080808080808080808B0
:100CC40008080808080808080808080808080808A0
:100CD4000808080808080808080808080808080890
:100CE4000808080808080808080808080808080880
:040CF40008080808DC
:00000001FF
